:100000000C9462000C948A000C948A000C948A0070
:100010000C948A000C948A000C948A000C948A0038
:100020000C948A000C948A000C948A000C948A0028
:100030000C948A000C948A000C948A000C948A0018
:100040000C94AB010C948A000C948A000C948A00E6
:100050000C948A000C948A000C948A000C948A00F8
:100060000C948A000C948A000000000023002600F3
:10007000290000000000240027002A0000000000E2
:10008000250028002B0004040404040404040202D4
:100090000202020203030303030301020408102007
:1000A0004080010204081020010204081020000012
:1000B0000008000201000003040700000000000027
:1000C0000000E20511241FBECFEFD8E0DEBFCDBF98
:1000D00011E0A0E0B1E0E8E7F0E102C005900D9288
:1000E000AE33B107D9F721E0AEE3B1E001C01D9214
:1000F000AC35B207E1F710E0C2E6D0E004C02197CA
:10010000FE010E943408C136D107C9F70E94F501EB
:100110000C943A080C940000833081F028F481306C
:1001200099F08230A9F008958730A9F08830C9F09D
:100130008430B1F4809180008F7D03C08091800075
:100140008F7780938000089584B58F7784BD08955C
:1001500084B58F7DFBCF8091B0008F778093B00006
:1001600008958091B0008F7DF9CF1F93CF93DF93D7
:10017000282F30E0F901E255FF4F8491F901E6564E
:10018000FF4FD491F901EA57FF4FC491CC23A9F056
:10019000162F81110E948C00EC2FF0E0EE0FFF1F54
:1001A000E458FF4FA591B4918FB7F894EC911111D9
:1001B00008C0D095DE23DC938FBFDF91CF911F91D4
:1001C0000895DE2BF8CFCF93DF9390E0FC01E65645
:1001D000FF4F24918A579F4FFC0184918823D1F0CF
:1001E00090E0880F991FFC01EE58FF4FA591B49144
:1001F000FC01E458FF4FC591D491623071F49FB770
:10020000F8943C91822F809583238C93E8812E2B48
:1002100028839FBFDF91CF9108958FB7F894EC9119
:100220002E2B2C938FBFF6CF8E50806480937C0052
:1002300080917A00806480937A0080917A0086FDB4
:10024000FCCF80917800909179000895CF93DF934F
:1002500096E0899FE0011124C050DF4F89818823F7
:1002600091F08A819B81AC81BD81481B590B6A0B3F
:100270007B0B453051056105710528F060E08881F0
:100280000E94B5001982DF91CF910895CF92DF923D
:10029000EF92FF92CF93DF936A017B0196E0899FF3
:1002A000E0011124C050DF4F61E088810E94B50059
:1002B00081E08983CA82DB82EC82FD82DF91CF916B
:1002C000FF90EF90DF90CF900895CF92DF92EF9262
:1002D000FF926B017C012BE83AE24AE25EE30E9466
:1002E000630687FD2EC02BE83AE24AEA5EE3C701C7
:1002F000B6010E94630687FD26C020ED3FE34FEF65
:100300005EE3C701B6010E94630687FD1EC02BE8AD
:100310003AE24AE25FE3C701B6010E94630687FD45
:1003200016C02DE235EB44E55FE3C701B6010E943C
:10033000630687FD0EC080E1FF90EF90DF90CF90C5
:10034000089581E0F9CF82E0F7CF83E0F5CF84E034
:10035000F3CF88E0F1CF1F920F920FB60F921124C6
:100360002F933F938F939F93AF93BF9380915801A7
:1003700090915901A0915A01B0915B0130915701C0
:1003800023E0230F2D3758F50196A11DB11D2093B1
:1003900057018093580190935901A0935A01B0934B
:1003A0005B018091530190915401A0915501B0914E
:1003B00056010196A11DB11D8093530190935401E4
:1003C000A0935501B0935601BF91AF919F918F912A
:1003D0003F912F910F900FBE0F901F90189526E818
:1003E000230F0296A11DB11DD2CFCF93DF93CDB7BE
:1003F000DEB768970FB6F894DEBF0FBECDBF789416
:1004000084B5826084BD84B5816084BD85B5826019
:1004100085BD85B5816085BD80916E0081608093CA
:100420006E00109281008091810082608093810033
:100430008091810081608093810080918000816043
:10044000809380008091B10084608093B10080919E
:10045000B00081608093B00080917A0084608093C6
:100460007A0080917A00826080937A0080917A008D
:10047000816080937A0080917A00806880937A000E
:100480001092C10062E084E00E94E30061E083E03A
:100490000E94E30061E081E10E94E30061E089E005
:1004A0000E94E30061E08AE00E94E30061E08BE0EB
:1004B0000E94E30060E083E00E94B50060E081E11B
:1004C0000E94B50060E089E00E94B50060E08AE02B
:1004D0000E94B50060E08BE00E94B5002FB7F89451
:1004E0008091580190915901A0915A01B0915B01FE
:1004F0002FBF80934F0190935001A0935101B0936F
:1005000052018FB7F8944090580150905901609073
:100510005A0170905B018FBF80914F019091500103
:10052000A0915101B0915201A3019201281B390BF6
:100530004A0B5B0BCA01B9010E94100720E030E0B2
:100540004AE754E40E9468066D837E838F83988710
:1005500040924F01509250016092510170925201AD
:10056000E2EBF0E08491EEE9F0E0F491F983EAE85F
:10057000F0E0F491F987FF2389F081110E948C004B
:100580002985E22FF0E0EE0FFF1FE859FF4FA591FC
:10059000B4918C913981382381E009F480E0109284
:1005A0004D0110924E0190914C01891751F08093AA
:1005B0004C0140924701509248016092490170926B
:1005C0004A018091470190914801A0914901B09161
:1005D0004A01B301A201481B590B6A0B7B0B8091A6
:1005E000430190914401A0914501B09146018417C7
:1005F0009507A607B707B0F490914B0180914C0185
:10060000981781F080934B01911103C021E0813054
:1006100009F020E020934D01913009F4811190E020
:1006200090934E0140914E0149838EE00E94140147
:10063000BC01990F880B990B0E94120720E030EC47
:100640004FE754E40E94680669877A878B879C8706
:100650008FE00E941401BC01990F880B990B0E9436
:10066000120720E030EC4FE754E40E9468066D87E3
:100670007E878F87988B80E10E941401BC01990FBF
:10068000880B990B0E94120720E030EC4FE754E4EE
:100690000E946806698B7A8B8B8B9C8B2091290139
:1006A00030912A0140912B0150912C016D817E8166
:1006B0008F8198850E94F7056B017C01C09229010A
:1006C000D0922A01E0922B01F0922C0159815523FE
:1006D00009F4A8C020911C0130911D0140911E0118
:1006E00050911F01209318013093190140931A0172
:1006F00050931B018090200190902101A090220135
:10070000B090230180921C0190921D01A0921E01C5
:10071000B0921F018091240190912501A0912601A2
:10072000B091270189839A83AB83BC838093200196
:1007300090932101A0932201B0932301C092240140
:10074000D0922501E0922601F092270180912801A4
:10075000843018F48F5F80932801809128018430C1
:1007600008F460C0C501B4010E94F6056D8B7E8B54
:100770008F8B988FA501940169817A818B819C81EF
:100780000E94F6059B01AC016D897E898F89988D49
:100790000E94F7054B015C0129813A814B815C8104
:1007A000C701B6010E94F6059B01AC01C501B40169
:1007B0000E94F70520E030E040E450E40E94680623
:1007C0006B017C0128E539E344E35CE30E946306A6
:1007D00087FF08C08AE0C82E87EDD82E83EAE82E6E
:1007E0008CE3F82EC0922D01D0922E01E0922F01C1
:1007F000F0923001109231011092320110923301C7
:100800001092340110923501109236011092370186
:10081000109238011092390110923A0110923B0166
:1008200010923C0180902D0190902E01A0902F01FC
:10083000B09030012DEB37E346E855E3C501B40134
:100840000E94C20720E030E0A901181654F4A50167
:10085000940160E070E080E89FE30E9468069B01DD
:10086000AC018091310190913201A0913301B0919E
:10087000340189839A83AB83BC836D817E818F81B0
:1008800098850E94C70729813A814B815C810E942B
:10089000F7056B017C011D8A20E030E040E85FE352
:1008A000C701B6010E94C20787FD0DC020E030E0FD
:1008B00040E85FE3C701B6010E94F6056B017C01C9
:1008C00091E09D8BE9CFC0923101D0923201E0924C
:1008D0003301F0923401AD890D89A1111CC020E0D3
:1008E00030E040E850E4C701B6010E94C7070E940B
:1008F000DA061B0120E030E040E850E469817A81AB
:100900008B819C810E94C7070E94DA0601E02616AF
:10091000370609F400E069857A858B859C850E94FD
:100920006501882339F1BD89B111C8C0682F70E015
:1009300090E080E00E94100769877A878B879C8708
:100940009B01AC01C701B6010E94C7070E94DA06ED
:100950007B0129853A854B855C8569817A818B810C
:100960009C810E94C7070E94DA06E1E0E983E6164F
:10097000F70609F419826D857E858F8598890E9416
:100980006501F82E69897A898B899C890E946501A5
:10099000382E6F2D70E090E080E00E941007A501D6
:1009A00094010E94C7076B017C012DEB37E346E8F9
:1009B00055E30E94630618160CF483C010E0632D03
:1009C00070E090E080E00E941007A50194010E9471
:1009D000C7076B017C012DEB37E346E855E30E9426
:1009E000630618160CF4ADC0F12C002329F0B301F6
:1009F000A20180E00E9446012981222329F0B3014F
:100A0000A20181E00E944601112329F0B301A20155
:100A100082E00E944601FF2029F0B301A20183E099
:100A20000E9446013D89332379F061E083E00E9412
:100A3000B50041E04093420140923E0150923F0197
:100A40006092400170924101B301A20180E00E94D6
:100A50002601B301A20181E00E942601B301A20197
:100A600082E00E942601B301A20183E00E942601D8
:100A7000809142018823D1F080913E0190913F0105
:100A8000A0914001B0914101A3019201281B390BB3
:100A90004A0B5B0BDA01C9010A97A105B10530F0D9
:100AA00060E083E00E94B5001092420140E050E017
:100AB000452B09F426CD0E94000023CDFD89F98342
:100AC0005ACFA70196016D817E818F8198850E9402
:100AD00068062091350130913601409137015091DF
:100AE00038010E94F7056B017C01C0923501D0925C
:100AF0003601E0923701F092380120E030E040E822
:100B00005FE30E94C20787FD59CF20E030E040E854
:100B10005FE3C701B6010E94F6056B017C0120E08E
:100B200030E040E85FE30E94C20787FFEECFC0924B
:100B30003501D0923601E0923701F092380111E090
:100B40003ECFA70196016D817E818F8198850E949D
:100B500068062091390130913A0140913B01509152
:100B60003C010E94F7056B017C01C0923901D092D3
:100B70003A01E0923B01F0923C0120E030E040E895
:100B80005FE30E94C20787FD2FCF20E030E040E8FE
:100B90005FE3C701B6010E94F6056B017C0120E00E
:100BA00030E040E85FE30E94C20787FFEECFC092CB
:100BB0003901D0923A01E0923B01F0923C01FF24CE
:100BC000F39413CFE3E4F1E082E390E0A0E0B0E03F
:100BD00080839183A283B383148215821682178245
:100BE00081E0808781871286138608955058BB273D
:100BF000AA270E940E060C9488070E947A0738F0F4
:100C00000E94810720F039F49F3F19F426F40C94D8
:100C100077070EF4E095E7FB0C947107E92F0E942B
:100C2000990758F3BA17620773078407950720F0EE
:100C300079F4A6F50C94BB070EF4E0950B2EBA2FB1
:100C4000A02D0B01B90190010C01CA01A0011124D2
:100C5000FF27591B99F0593F50F4503E68F11A167E
:100C6000F040A22F232F342F4427585FF3CF46950F
:100C700037952795A795F0405395C9F77EF41F1631
:100C8000BA0B620B730B840BBAF09150A1F0FF0FFB
:100C9000BB1F661F771F881FC2F70EC0BA0F621FE7
:100CA000731F841F48F4879577956795B795F795D7
:100CB0009E3F08F0B0CF9395880F08F09927EE0F6C
:100CC0009795879508950E944D0708F481E008954F
:100CD0000E947C060C9488070E94810758F00E94AD
:100CE0007A0740F029F45F3F29F00C947107511105
:100CF0000C94BC070C9477070E94990768F399231A
:100D0000B1F3552391F3951B550BBB27AA27621707
:100D10007307840738F09F5F5F4F220F331F441F14
:100D2000AA1FA9F335D00E2E3AF0E0E832D0915048
:100D30005040E695001CCAF72BD0FE2F29D0660F35
:100D4000771F881FBB1F261737074807AB07B0E878
:100D500009F0BB0B802DBF01FF2793585F4F3AF07E
:100D60009E3F510578F00C9471070C94BC075F3FCF
:100D7000E4F3983ED4F3869577956795B795F79504
:100D80009F5FC9F7880F911D9695879597F90895EC
:100D9000E1E0660F771F881FBB1F62177307840788
:100DA000BA0720F0621B730B840BBA0BEE1F88F797
:100DB000E09508950E94E1066894B1110C94BC0777
:100DC00008950E94A10788F09F5798F0B92F99279E
:100DD000B751B0F0E1F0660F771F881F991F1AF026
:100DE000BA95C9F714C0B13091F00E94BB07B1E0C9
:100DF00008950C94BB07672F782F8827B85F39F0C8
:100E0000B93FCCF3869577956795B395D9F73EF4BE
:100E100090958095709561957F4F8F4F9F4F089566
:100E2000E89409C097FB3EF4909580957095619584
:100E30007F4F8F4F9F4F9923A9F0F92F96E9BB273A
:100E40009395F695879577956795B795F111F8CFB6
:100E5000FAF4BB0F11F460FF1BC06F5F7F4F8F4F21
:100E60009F4F16C0882311F096E911C0772321F017
:100E70009EE8872F762F05C0662371F096E8862FAF
:100E800070E060E02AF09A95660F771F881FDAF706
:100E9000880F9695879597F90895990F0008550F33
:100EA000AA0BE0E8FEEF16161706E807F907C0F0F0
:100EB00012161306E407F50798F0621B730B840BF8
:100EC000950B39F40A2661F0232B242B252B21F4D2
:100ED00008950A2609F4A140A6958FEF811D811D72
:100EE000089597F99F6780E870E060E008959FEFAC
:100EF00080EC089500240A941616170618060906B1
:100F0000089500240A94121613061406050608957F
:100F1000092E0394000C11F4882352F0BB0F40F407
:100F2000BF2B11F460FF04C06F5F7F4F8F4F9F4F47
:100F3000089557FD9058440F551F59F05F3F71F0C9
:100F40004795880F97FB991F61F09F3F79F0879530
:100F50000895121613061406551FF2CF4695F1DFB9
:100F600008C0161617061806991FF1CF8695710549
:100F7000610508940895E894BB2766277727CB017D
:100F800097F908950E944D0708F48FEF08950E9485
:100F9000DA070C9488070E947A0738F00E948107CC
:100FA00020F0952311F00C9471070C94770711240D
:100FB0000C94BC070E94990770F3959FC1F3950F9D
:100FC00050E0551F629FF001729FBB27F00DB11DCD
:100FD000639FAA27F00DB11DAA1F649F6627B00D5D
:100FE000A11D661F829F2227B00DA11D621F739F46
:100FF000B00DA11D621F839FA00D611D221F749F54
:101000003327A00D611D231F849F600D211D822F9A
:10101000762F6A2F11249F5750409AF0F1F08823C1
:101020004AF0EE0FFF1FBB1F661F771F881F9150EE
:101030005040A9F79E3F510580F00C9471070C9425
:10104000BC075F3FE4F3983ED4F3869577956795A8
:10105000B795F795E7959F5FC1F7FE2B880F911D18
:101060009695879597F90895EE0FFF1F0590F491D7
:08107000E02D0994F894FFCF74
:101078001100000000000900000000000A00000044
:1010880000000B000000000000000000000000004D
:101098000000000000000000000000000000000048
:0E10A8003F00000000000000000000000000FB
:00000001FF
